:020000040000fa
:080000000002040000000000f2
:020000040000fa
:040008009a03000057
:020000040000fa
:04000c00b403000039
:020000040000fa
:040010006603000083
:020000040000fa
:04001400ce03000017
:020000040000fa
:04001800e8030000f9
:020000040000fa
:04001c0032030000ab
:020000040000fa
:040020008003000059
:020000040000fa
:040024004c03000089
:020000040000fa
:040028003c04000094
:020000040000fa
:04002c003c04000090
:020000040000fa
:040030003c0400008c
:020000040000fa
:040034003c04000088
:020000040000fa
:040038003c04000084
:020000040000fa
:04003c003c04000080
:020000040000fa
:040040003c0400007c
:020000040000fa
:040044003c04000078
:020000040000fa
:040048003c04000074
:020000040000fa
:04004c003c04000070
:020000040000fa
:040050003c0400006c
:020000040000fa
:040054003c04000068
:020000040000fa
:040058003c04000064
:020000040000fa
:04005c003c04000060
:020000040000fa
:040060003c0400005c
:020000040000fa
:040064003c04000058
:020000040000fa
:040068003c04000054
:020000040000fa
:04006c003c04000050
:020000040000fa
:040070003c0400004c
:020000040000fa
:040074003c04000048
:020000040000fa
:040078003c04000044
:020000040000fa
:04007c003c04000040
:020000040000fa
:040080003c0400003c
:020000040000fa
:040084003c04000038
:020000040000fa
:040088003c04000034
:020000040000fa
:04008c003c04000030
:020000040000fa
:040090003c0400002c
:020000040000fa
:040094003c04000028
:020000040000fa
:040098003c04000024
:020000040000fa
:04009c003c04000020
:020000040000fa
:0400a0003c0400001c
:020000040000fa
:0400a4003c04000018
:020000040000fa
:0400a8003c04000014
:020000040000fa
:0400ac003c04000010
:020000040000fa
:0400b0003c0400000c
:020000040000fa
:0400b4003c04000008
:020000040000fa
:0400b8003c04000004
:020000040000fa
:0400bc003c04000000
:020000040000fa
:0400c0003c040000fc
:020000040000fa
:0400c4003c040000f8
:020000040000fa
:0400c8003c040000f4
:020000040000fa
:0400cc003c040000f0
:020000040000fa
:0400d0003c040000ec
:020000040000fa
:0400d4003c040000e8
:020000040000fa
:0400d8003c040000e4
:020000040000fa
:0400dc003c040000e0
:020000040000fa
:0400e0003c040000dc
:020000040000fa
:0400e4003c040000d8
:020000040000fa
:0400e8003c040000d4
:020000040000fa
:0400ec003c040000d0
:020000040000fa
:0400f0003c040000cc
:020000040000fa
:0400f4003c040000c8
:020000040000fa
:0400f8003c040000c4
:020000040000fa
:0400fc003c040000c0
:020000040000fa
:040100003c040000bb
:020000040000fa
:040104003c040000b7
:020000040000fa
:040108003c040000b3
:020000040000fa
:04010c003c040000af
:020000040000fa
:040110003c040000ab
:020000040000fa
:040114003c040000a7
:020000040000fa
:040118003c040000a3
:020000040000fa
:04011c003c0400009f
:020000040000fa
:040120003c0400009b
:020000040000fa
:040124003c04000097
:020000040000fa
:040128003c04000093
:020000040000fa
:04012c003c0400008f
:020000040000fa
:040130003c0400008b
:020000040000fa
:040134003c04000087
:020000040000fa
:040138003c04000083
:020000040000fa
:04013c003c0400007f
:020000040000fa
:040140003c0400007b
:020000040000fa
:040144003c04000077
:020000040000fa
:040148003c04000073
:020000040000fa
:04014c003c0400006f
:020000040000fa
:040150003c0400006b
:020000040000fa
:040154003c04000067
:020000040000fa
:040158003c04000063
:020000040000fa
:04015c003c0400005f
:020000040000fa
:040160003c0400005b
:020000040000fa
:040164003c04000057
:020000040000fa
:040168003c04000053
:020000040000fa
:04016c003c0400004f
:020000040000fa
:040170003c0400004b
:020000040000fa
:040174003c04000047
:020000040000fa
:040178003c04000043
:020000040000fa
:04017c003c0400003f
:020000040000fa
:040180003c0400003b
:020000040000fa
:040184003c04000037
:020000040000fa
:040188003c04000033
:020000040000fa
:04018c003c0400002f
:020000040000fa
:040190003c0400002b
:020000040000fa
:040194000204000061
:020000040000fa
:040198003c04000023
:020000040000fa
:04019c003c0400001f
:020000040000fa
:0401a0003c0400001b
:020000040000fa
:0401a4003c04000017
:020000040000fa
:0401a8003c04000013
:020000040000fa
:0401ac003c0400000f
:020000040000fa
:0401b0003c0400000b
:020000040000fa
:0401b4003c04000007
:020000040000fa
:0401b8003c04000003
:020000040000fa
:0401bc003c040000ff
:020000040000fa
:0401c0003c040000fb
:020000040000fa
:0401c4003c040000f7
:020000040000fa
:0401c8003c040000f3
:020000040000fa
:0401cc003c040000ef
:020000040000fa
:0401d0003c040000eb
:020000040000fa
:0401d4003c040000e7
:020000040000fa
:0401d8003c040000e3
:020000040000fa
:0401dc003c040000df
:020000040000fa
:0401e0003c040000db
:020000040000fa
:0401e4003c040000d7
:020000040000fa
:0401e8003c040000d3
:020000040000fa
:0401ec003c040000cf
:020000040000fa
:0401f0003c040000cb
:020000040000fa
:0401f4003c040000c7
:020000040000fa
:0401f8003c040000c3
:020000040000fa
:0401fc003c040000bf
:020000040000fa
:040200003c040000ba
:020000040000fa
:040204003c040000b6
:020000040000fa
:040208003c040000b2
:020000040000fa
:04020c003c040000ae
:020000040000fa
:040210003c040000aa
:020000040000fa
:040214003c040000a6
:020000040000fa
:040218003c040000a2
:020000040000fa
:04021c003c0400009e
:020000040000fa
:040220003c0400009a
:020000040000fa
:040224003c04000096
:020000040000fa
:040228003c04000092
:020000040000fa
:04022c003c0400008e
:020000040000fa
:040230003c0400008a
:020000040000fa
:040234003c04000086
:020000040000fa
:040238003c04000082
:020000040000fa
:04023c003c0400007e
:020000040000fa
:040240003c0400007a
:020000040000fa
:040244003c04000076
:020000040000fa
:040248003c04000072
:020000040000fa
:04024c003c0400006e
:020000040000fa
:040250003c0400006a
:020000040000fa
:040254003c04000066
:020000040000fa
:040258003c04000062
:020000040000fa
:04025c003c0400005e
:020000040000fa
:040260003c0400005a
:020000040000fa
:040264003c04000056
:020000040000fa
:040268003c04000052
:020000040000fa
:04026c003c0400004e
:020000040000fa
:040270003c0400004a
:020000040000fa
:040274003c04000046
:020000040000fa
:040278003c04000042
:020000040000fa
:04027c003c0400003e
:020000040000fa
:040280003c0400003a
:020000040000fa
:040284003c04000036
:020000040000fa
:040288003c04000032
:020000040000fa
:04028c003c0400002e
:020000040000fa
:040290003c0400002a
:020000040000fa
:040294003c04000026
:020000040000fa
:040298003c04000022
:020000040000fa
:04029c003c0400001e
:020000040000fa
:0402a0003c0400001a
:020000040000fa
:0402a4003c04000016
:020000040000fa
:0402a8003c04000012
:020000040000fa
:0402ac003c0400000e
:020000040000fa
:0402b0003c0400000a
:020000040000fa
:0402b4003c04000006
:020000040000fa
:0402b8003c04000002
:020000040000fa
:0402bc003c040000fe
:020000040000fa
:0402c0003c040000fa
:020000040000fa
:0402c4003c040000f6
:020000040000fa
:0402c8003c040000f2
:020000040000fa
:0402cc003c040000ee
:020000040000fa
:0402d0003c040000ea
:020000040000fa
:0402d4003c040000e6
:020000040000fa
:0402d8003c040000e2
:020000040000fa
:0402dc003c040000de
:020000040000fa
:0402e0003c040000da
:020000040000fa
:0402e4003c040000d6
:020000040000fa
:0402e8003c040000d2
:020000040000fa
:0402ec003c040000ce
:020000040000fa
:0402f0003c040000ca
:020000040000fa
:0402f4003c040000c6
:020000040000fa
:0402f8003c040000c2
:020000040000fa
:0402fc003c040000be
:020000040000fa
:040300003c040000b9
:020000040000fa
:040304003c040000b5
:020000040000fa
:040308003c040000b1
:020000040000fa
:04030c003c040000ad
:020000040000fa
:040310003c040000a9
:020000040000fa
:040314003c040000a5
:020000040000fa
:040318003c040000a1
:020000040000fa
:04031c003c0400009d
:020000040000fa
:040320003c04000099
:020000040000fa
:040324003c04000095
:020000040000fa
:100400006f3921002efd22000e018800000000003f
:10041000000020000000e000020032000001200087
:100420002002880014000700150107000000e0000a
:1004300003003a00e0ed2100010020000200370037
:100440000000200001002000810f70000100320038
:100450000f000700000020000000e0000200320052
:1004600000000200000000009024020000000000d4
:100470000040da000000fe00200020000000e00044
:1004800002003200100020009001880000000600e9
:10049000a1028800800478000000eb001f003700f4
:1004a000e284440054a0b4009905ba00e2844400f8
:1004b00054a0b4009906ba00e284440054a0b400e9
:1004c0000006eb00476fde00fd07b200ae018800ba
:1004d000636ce10003003a000ad801000000eb0061
:1004e0000e003700606ce10008003a00004deb00a0
:1004f0000a05e800020039003420ec000af0a000f0
:100500008b05e900f9ff3e00040037006168e10057
:10051000010032000086eb000b00070019c7ba008b
:100520001905ba000e04e00003003a000a00e000da
:10053000dbff3a0000000600fe07b200ae028800b2
:100540008a047800f5ff37000cd0a300e20f4d00bd
:100550001c00390089027800354dba000a05e80010
:10056000020039003420ec000af0a0008b05e900fd
:100570000f003200254dba000a05e80002003900dc
:100580003420ec000af0a0008b05e90008003200de
:100590000c00e0000600320015cdba000a05e800a4
:1005a000020039003420ec000af0a0008b05e900bd
:1005b0008984e80054a0b4000b00e000e2ff3a0098
:1005c000000006009902ba00055d78008b05e9007d
:1005d000f7ff3200c82ade00055d78008b05e900d0
:1005e000f3ff32000c00e000f1ff320019ddba0029
:1005f000eeff3700000000000000000000000000d7
:1006000000000000000000000000000000000000ea
:1006100000000000000000000000000000000000da
:1006200000000000000000000000000000000000ca
:1006300000000000000000000000000000000000ba
:1006400000000000000000000000000000000000aa
:10065000000000000000000000000000000000009a
:10066000000000003600f800809fbe00829fbe00a0
:10067000849fbe00869fbe0000082000c0130700b4
:100680004f03be004f02be004f01be004f00be0030
:100690003600f900004006003600f800809fbe00da
:1006a000829fbe00849fbe00869fbe00000820007f
:1006b000b31307004f03be004f02be004f01be0040
:1006c0004f00be003600f900004006003600f8007a
:1006d000809fbe00829fbe00849fbe00869fbe009a
:1006e00000042000a61307004f03be004f02be0007
:1006f0004f01be004f00be003600f900004006006a
:100700003600f800809fbe00829fbe00849fbe001e
:10071000869fbe0000022000991307004f03be0011
:100720004f02be004f01be004f00be003600f90070
:10073000004006003600f800809fbe00829fbe0089
:10074000849fbe00869fbe00100020008c1307000f
:100750004f03be004f02be004f01be004f00be005f
:100760003600f900004006003600f800809fbe0009
:10077000829fbe00849fbe00869fbe002000200096
:100780007f1307004f03be004f02be004f01be00a3
:100790004f00be003600f900004006003600f800a9
:1007a000809fbe00829fbe00849fbe00869fbe00c9
:1007b00040002000721307004f03be004f02be002e
:1007c0004f01be004f00be003600f9000040060099
:1007d0003600f800809fbe00829fbe00849fbe004e
:1007e000869fbe0080002000651307004f03be00f7
:1007f0004f02be004f01be004f00be003600f900a0
:10080000004006003600f8003200f8003400f8001e
:1008100010002000a0018800100020009001880036
:1008200023cea800800921001010a000a18c800018
:10083000708c800001000100418d8000108d8000cf
:1008400001000100e18d8000b08d800001000100f9
:100850000000000000000000000000000000000098
:100860000b68a90023cea9003400f9003200f9007a
:100870003600f900004006000040da000000fe00eb
:04088000000005006f
:020000040000fa
:100884001000fa00889fbe000004780010002000c9
:10089400e0b79f000000eb00f0b79f006000b800d5
:1008a40080bf9f0091bf9f00a0bf9f00b1bf9f006a
:1008b400c0bf9f00d1bf9f001800e00002003d00b0
:1008c4001838a30014003a00980078006180600092
:1008d4000004e0000d003a000000eb001004980052
:1008e400180090008000eb00e90f5000e08f5800e2
:1008f400100036000000eb00100498006fb0970061
:100904004f04be000080fa00000006001000200022
:1009140010049800f2ff37001878a300f0ff3200ab
:1009240098007800618060000004e000f7ff3a005e
:10093400e9ff3700000601003901370016013700ce
:10094400fc003700e90037005f0037004100370042
:10095400360037001e00370001003700420137001f
:10096400b810900068b09000808f50008d02320063
:100974001880a000b810900068b09000808f5000dc
:100984009e013900b810900068b09000808f50002c
:10099400daff360068b090009810900000804000a4
:1009a40060b49800e8b0900038109000808f500038
:1009b400d2ff36003810900060b498006fb09700f2
:1009c4004f04be000080fa0000000600cfff37008d
:1009d4001880a00068009000f80090000001e80072
:1009e40062049800810f5000c4ff3600800020008c
:1009f40010049800780090000000e800600498005b
:100a040028e091000004e000bcff3200200e20002a
:100a140008004000801107006fb097004f04be002b
:100a24000080fa0000000600b8ff3700281090008c
:100a3400e20f5000a801320038b89000a8b8900026
:100a440010219000112098007000200010049800dc
:100a5400aaff37001880a00038b89000104090001a
:100a64000078a300b701320008109000981090009d
:100a740000804000001498008810900068b0900036
:100a8400808f50009dff360068b0900000149800dd
:100a940038b89000c10e20008880400010119000ea
:100aa40011109800281090000000e000e6ff3200ca
:100ab40028109000e20f500090ff3a0060002000e0
:100ac400100498008dff37001880a0000000eb0090
:100ad40000149800e0032000400c980038b89000ff
:100ae400010220008880400010119000111098002d
:100af400181890000014980028109000e20f50007d
:100b0400a60132009818900058209000808f500061
:100b1400e9003200a818900078289000808f5000d7
:100b2400e5003200d8289000281990007828900019
:100b3400000051000100b80080bf9f0091bf9f00da
:100b44000fb897009fb897006829900070011100b2
:100b54000201e900030033008100d1000080d300ca
:100b6400fbff370080bf9f0091bf9f00b82090001b
:100b74001819900058209000000051000100b8009e
:100b8400a0bf9f00b1bf9f002fb89700bfb89700c8
:100b940048219000700111000201e90003003300b4
:100ba4008100d1000080d300fbff3700a0bf9f006d
:100bb400b1bf9f00389190000fb897009fb897007d
:100bc4000200b800c0bf9f00d1bf9f002fb997009b
:100bd400bfb997004fba9700dfba97000500090024
:100be40042aad8008000eb00c0bf9f00d1bf9f0085
:100bf4002fb99700bfb997000fb897009fb8970017
:100c0400800f5100818f5900ec013600389090001c
:100c14004fb99700dfb997008000eb000200500045
:100c240083805800c0bf9f00d1bf9f00081190006f
:100c340098109000200320000088b90000004100b3
:100c440000149800281090000000e000a1003a0071
:100c540018b990004fb89700dfb89700cf91de0025
:100c6400800f5100818f5900c201360018b89000de
:100c7400cf80de00c0bf9f00d1bf9f00f8b99000b5
:100c84004fba9700dfba970038b890000401780093
:100c94008000eb000300010038b89000a0509000e1
:100ca4008180fb00305090004800dd00008070001f
:100cb4004fb99700dfb997000208780038b8900060
:100cc400a05890008180fb00305890004800dd005f
:100cd400008070004fb99700dfb9970002087800d0
:100ce400500020001004980004ff37001880a00072
:100cf40028009000b80090000001e8002204980049
:100d0400810f5000fdfe3600380090000000e8001e
:100d140020049800400020001848a300f6fe3a0082
:100d24006fb097004f04be000080fa000000060078
:100d3400f6fe37001880a1001800e00003003d0013
:100d440018e8a3000100320018d0a00008d89100d0
:100d54000004e00008013a001800e000e7fe3d004e
:100d640018d8a300e5fe32001818a300e3fe3200f1
:100d74001828a300e1fe32001878a300dffe3a0031
:100d84001848a300ddfe320018d0a1003000200076
:100d940010049800d9fe37001880a00008007800dd
:100da4002f0f0700efb0970001006000e0b79f002d
:100db400b8b89000114090000074a10090409800d1
:100dc400d8b8900038b890000100010038b89000fd
:100dd400205190000281fb00b0509000c808dd0053
:100de4008100710038b8900000c190000281fb00be
:100df40010c090004800dd0082087000e08580008b
:100e0400e20f5000ec00320028e091000004e00002
:100e140089003a002000200010049800b7fe370033
:100e24001880a0000000eb002004980060049800e3
:100e34001830a1001810a1001898a3006d0032000a
:100e44001840a10028e091000004e00003003200f3
:100e5400200e20000800400097100700100020001a
:100e640010049800a5fe370008007800040e07005f
:100e7400efb0970001006000e0b79f00b8b89000a1
:100e8400114090000074a100904098002810900038
:100e9400e20f50006d003200380090000000e800be
:100ea40020049800780090000000e8006004980096
:100eb40010002000eaff3700689090008000eb00eb
:100ec400c0bf9f00d1bf9f00281090000000e00029
:100ed4005fff320028109000e20f500080ff3a00bc
:100ee4000000eb00f0b79f0010868000ffb0970071
:100ef400808f50007aff31007fb097007400b900f2
:100f04006010b000680178004fb89700dfb8970010
:100f1400cf91de00800f5100818f5900030136000c
:100f24007fb097007400b9006010b00068007800ca
:100f3400cf80de00c0bf9f00d1bf9f007fb097006d
:100f44007400b9002011b000e80178004fba97008e
:100f5400dfba97007fb097007400b900a010b0000a
:100f640068007800040178008000eb0003000100b1
:100f74007fb097007400b900a010b000680078003a
:100f8400a05090008180fb00305090004800dd00ac
:100f9400008070004fb99700dfb99700020878000d
:100fa4007fb097007400b900a010b000680078000a
:100fb400a05890008180fb00305890004800dd006c
:100fc400008070004fb99700dfb9970002087800dd
:100fd4007fb097000000e800f0b79f001186800002
:100fe4007fb09700808f5000c3ff3e005000200068
:100ff4003cff37001840a00092ff3700e8b0900093
:10100400181090000080500060b49800e8b0900080
:1010140038109000808f500038fe3100b8109000d6
:1010240061b498006fb097004f04be000080fa00ce
:101034000000060035fe3700200e200008004000a6
:101044001d1007002000200073ff37000000eb0094
:10105400f0b79f0058109000ffb09700808f5000a9
:101064008dff31007fb097007400b900a010b0006c
:10107400e8007800114090000074a10090409800ae
:101084007fb097000000e800f0b79f00d8109000f0
:101094007fb09700808f50007fff36007fb09700ad
:1010a4007400b900a010b000e8007800114090006e
:1010b4000074a100904098007fb097000000e80001
:1010c400f0b79f00d81090007fb09700808f500039
:1010d400e4ff3e0070ff37001880a00038b890008d
:1010e400a0c090008180fb0030c190004811dd0059
:1010f40002817000d8089000810041001021900006
:101104001120980038b8900020c190000281fb00a3
:10111400b0c09000c808dd00810071005033200089
:10112400808f5000f5fd36000000e80020bc9800d8
:1011340038b89000a8b890001021900011209800b1
:1011440041fe370008007800880e0700efb09700d2
:1011540001006000e0b79f00281090000000e0004c
:10116400a1003a00b8b89000114090000074a000ab
:10117400904098003cfe3700dd890a00180000000a
:10118400800d200008004000f30f070080c46400b5
:10119400dd090a0018000000effe3700c8089000bf
:1011a40021bc980038b89000a8b890001021900095
:1011b4001120980053fe37000000eb00f0b79f00a9
:1011c40010868000ffb09700808f50000eff310022
:1011d4007fb097007400b900a010b000e800780058
:1011e400114090000074a100904098007fb09700d7
:1011f4007400b900e010b000e80078007fb19700f7
:101204007411b900a01020000200400068007800aa
:10121400010001007fb097007400b900a010b00075
:1012240068007800205190000281fb00b0509000cb
:10123400c808dd00810071007fb197007411b90006
:10124400a0102000020040006800780000c1900057
:101254000281fb0010c090004800dd00820870008d
:101264007fb097000000e800f0b79f00118680006f
:101274007fb09700808f5000e3fe36007fb0970068
:101284007400b900a010b000e8007800114090008c
:101294000074a100904098007fb097007400b900da
:1012a400e010b000e80078007fb197007411b90035
:1012b400a010200002004000680078000100010036
:1012c4007fb097007400b900a010b00068007800e7
:1012d400205190000281fb00b0509000c808dd004e
:1012e400810071007fb197007411b900a010200033
:1012f400020040006800780000c190000281fb00f9
:1013040010c090004800dd00820870007fb0970094
:101314000000e800f0b79f00118680007fb09700be
:10132400808f5000aaff3e00b7fe37007fb09700c1
:101334007400b9008010b000680178004fb89700bd
:10134400dfb897008001eb00800f5100818f5900b6
:10135400fafe31007fb097007400b9008010b0002d
:10136400680078008000eb00c0bf9f00d1bf9f00e1
:10137400f2fe370028b990004fb89700dfb8970005
:101384008001eb00800f5100818f59003bfe31003a
:1013940028b890008000eb00c0bf9f00d1bf9f0021
:1013a40036fe37001880a1006fb097004f04be00ce
:1013b4000080fa000000060054fd37006890900099
:1013c4008000eb00c0bf9f00d1bf9f0008119000b8
:1013d40098109000200320000088b900000041000c
:1013e4000014980017fe370028109000e20f5000f8
:1013f4009dfd3a00b8b89000114090000074a00020
:10140400904098000000eb00f0b79f00d8109000c7
:101414007fb09700808f500093fd36007fb0970017
:101424007400b900a010b000e800780011409000ea
:101434000074a000904098007fb097000000e8007e
:04144400f1ff37007d
:020000040000fa
:10144800f6874700889fbe008a9fbe008c9fbe001b
:101458008e1f780010002000f0af9f006a1821004e
:101468000000eb00000d7800219f2000218c8800ef
:1014780064074500a1cc2f00010f7800e60645005f
:1014880061332000810e7800408c88006804450094
:10149800001c2100000c78008880e800027b2100f5
:1014a8008208780002d22100a28c880082d821000c
:1014b800928c880002da2100b28c880091007800b2
:1014c800010001001800780001c12000f90f200078
:1014d8002041900021409800c808de00304190006b
:1014e80031409800180078009a0078004001900078
:1014f8004100980018007800c0409000f0400a00b1
:10150800010500004140980018007800e040900074
:1015180082c5b30062409800f0409000e1c5b30076
:101528007140980018007800a0499000f0400a0027
:1015380003000000234898001800780080519000ac
:10154800f0400a00030000000350980018007800db
:10155800c0499000f0400a00030500004348980085
:1015680018007800e049900062489800704990009f
:101578007148980018007800ea0044000982600069
:101588002051900024509800c809de003051900086
:10159800335098001800780000599000f0400a0075
:1015a800020000000258980018007800405190008e
:1015b800f0400a000200000042509800180078002d
:1015c8006051900080c5eb006b50980070519000fe
:1015d800fac7b3007a509800180078007e064400d5
:1015e80009016600a2b79f0020599000cfe3970039
:1015f800275898004861de0092b79f003059900044
:10160800afe3970037589800180078000061900001
:10161800f0400a00020000000260980018007800fc
:1016280040599000f0400a0002000000425898001b
:1016380018007800605990006b5898007059900015
:101648007a5898001800780002f32f00080141002a
:101658008902610020639000256098004811de002f
:10166800b062900032609800180078001e0178007f
:101678008022900002209800180078001d01780050
:1016880090229000122098001800780040c1900025
:10169800f0400a000200000042c0980018007800dc
:1016a80060c19000f0400a000200000062c098008b
:1016b8001800780000c99000f0400a0002000000fd
:1016c80002c898001800780020c99000f0400a006d
:1016d8000200000022c898001800780040c9900055
:1016e800f0400a000200000042c898001800780084
:1016f80060c99000f0400a000200000062c898002b
:1017080018007800c2f32f00080141008902610027
:1017180000d3900005d098004811de0090d29000c8
:1017280012d098001800780040d19000f0400a00cc
:101738000200000042d098001800780060d19000a4
:10174800f0400a000200000062d0980018007800fb
:1017580000d99000f0400a000200000002d898006a
:101768001800780020d99000f0400a00020000001c
:1017780022d898001800780040e19000f0400a0054
:101788000200000042e098001800780060e1900034
:10179800f0400a000200000062e09800180078009b
:1017a80000e99000f0400a000200000002e89800fa
:1017b8001800780020e99000f0400a0002000000bc
:1017c80022e8980018017800124090000074a100e7
:1017d8001041980018017800124090000054a100b0
:1017e8001041980018017800124090000044a100b0
:1017f8001041980018017800124090000064a10080
:1018080010419800180078001004a1001800780012
:101818001014a10018017800124090000034a100b3
:1018280010419800ec0244000d8020008d0a7800d9
:10183800e0032000800878007001440007142000ad
:1018480007097800f2004400009021008008780021
:101858007207470007692000070f780074044400e6
:10186800c0222100000c780064834000478e2100cc
:10187800070b7800671e2200478d8800c7252200c5
:10188800378d880047272200578d88001603780077
:10189800f1b79f00e2b79f00c3b79f00b4b79f009e
:1018a800d5b79f000600010018007800c6c02000c8
:1018b8008903630087bf9f00a04390008ff39700c0
:1018c800274098004833de00b04390003640980027
:1018d80018007800dfb29700950278004003900066
:1018e8004500980018007800c0429000f0400a00b7
:1018f800050400004540980018007800e042900078
:101908006b409800f04290007a40980018007800e8
:10191800a04a9000f0400a00050000002548980001
:101928001800780080529000f0400a00050000007e
:101938000550980018007800c04a9000f0400a004e
:10194800050000004548980018007800e04a90001b
:10195800f0400a000500000065489800180078006b
:101968004538200009836200a05390002650980053
:10197800c82ade00305390003550980018007800cf
:10198800805a9000f0400a000500000005589800b1
:1019980018007800c0529000f0400a0005000000ce
:1019a8004550980018007800e05290006b5098005d
:1019b800f05290007a50980018007800a05a9000d1
:1019c800f0400a000500000025589800180078002b
:1019d80080629000f0400a00050000000560980051
:1019e80018007800c05a9000f0400a000500000076
:1019f8004558980018007800e05a90006b589800f5
:101a0800f05a90007a58980018007800a062900068
:101a18003fb297002460980030629000cfb19700e1
:101a280033609800180078006fb1970012017800b1
:101a3800802190000220980018007800ffb09700dd
:101a4800910078001021900011209800180078006b
:101a5800c0c09000f0400a000100000041c098009a
:101a680018007800e0c09000f0400a000100000073
:101a780061c0980018007800a13820000981600032
:101a880080c9900002c89800c808de0010c99000fc
:101a980011c89800180078009e0078005021900026
:101aa800512098001800780021f22f00888040000b
:101ab8000981600080d1900002d09800c808de003b
:101ac80010d1900011d0980018007800c0d0900074
:101ad800f0400a000100000041d09800180078008a
:101ae800e0d09000f0400a000100000061d09800aa
:101af8001800780080d89000f0400a00010000002b
:101b080001d8980018007800a0d89000f0400a008a
:101b18000100000021d8980018007800c0e090006b
:101b2800f0400a000100000041e098001800780029
:101b3800e0e09000f0400a000100000061e0980039
:101b48001800780080e89000f0400a0001000000ca
:101b580001e8980018007800a0e89000f0400a001a
:101b68000100000021e898009800780011409000da
:101b78000074a100904098009800780011409000ef
:101b88000054a100904098009800780011409000ff
:101b98000044a100904098009800780011409000ff
:101ba8000064a00090409800180078001004a1007c
:101bb800180078001014a1009800780011409000d7
:101bc8000034a10090409800720747000d0f78007c
:101bd800e0032000000e7800f0004400021420000a
:101be80082087800f206440007902100870e7800ea
:101bf8006406460000692000000e78007404440062
:101c080080292100000c78006681400063a0210033
:101c18000309780043292200e38d8800a3302200bd
:101c2800d38d880023322200f38d880012017800ba
:101c3800f1b79f000200010018007800e2c0200000
:101c48008901610020429000234098004811de007d
:101c5800b041900032409800180078001e017800ca
:101c6800c0019000420098001800780040419000a0
:101c7800f0400a0002040000424098001800780072
:101c8800604190006b409800704190007a40980045
:101c98001800780020499000f0400a000200000077
:101ca800224898001800780000519000f0400a007f
:101cb8000200000002509800180078004049900087
:101cc800f0400a000200000042489800180078001e
:101cd80060499000f0400a00020000006248980045
:101ce80018007800023f200089016100205290000e
:101cf800235098004811de00b051900032509800ef
:101d08001800780000599000f0400a000200000016
:101d1800025898001800780040519000f0400a00de
:101d280002000000425098001800780060519000ae
:101d38006b509800705190007a5098001800780005
:101d480020599000f0400a00020000002258980034
:101d58001800780000619000f0400a0002000000be
:101d6800026098001800780040599000f0400a007e
:101d7800020000004258980018007800605990004e
:101d88006b589800705990007a589800180078009d
:101d9800206190004fe19700226098003061900028
:101da800afe397003760980018007800ffb09700fd
:101db8009100780000219000012098001800780018
:101dc8009d007800102190001120980018007800dc
:101dd800c0c09000f0400a000100000041c0980017
:101de80018007800e0c09000f0400a0001000000f0
:101df80061c0980018007800613f200009816000e8
:101e080080c9900002c89800c808de0010c9900078
:101e180011c89800180078009c00780050219000a4
:101e2800512098001800780001f12f0088804000a8
:101e38008984600000d1900009d09800c808de00ad
:101e480010d1900011d0980018007800c0d09000f0
:101e5800f0400a000100000041d098001800780006
:101e6800e0d09000f0400a000100000061d0980026
:101e78001800780080d89000f0400a0001000000a7
:101e880001d8980018007800a0d89000f0400a0007
:101e98000100000021d8980018007800c0e09000e8
:101ea800f0400a000100000041e0980018007800a6
:101eb800e0e09000f0400a000100000061e09800b6
:101ec8001800780080e89000f0400a000100000047
:101ed80001e8980018007800a0e89000f0400a0097
:101ee8000100000021e89800980078001140900057
:101ef8000074a1009040980098007800114090006c
:101f08000054a1009040980098007800114090007b
:101f18000044a1009040980098007800114090007b
:101f28000064a00090409800180078001004a100f8
:101f3800180078001014a100980078001140900053
:101f48000034a100904098007fa897004f077800c0
:101f58004f06be004f05be004f04be006f01b10022
:041f6800000006006f
:020000040000fa
:101f6c000800fa00889fbe008a9fbe001100200066
:101f7c0081bf9f008000eb0091bf9f0091bf9f002d
:101f8c00501190009fb89700810f5100230136002b
:101f9c00a532200007362000858353008783d100ab
:101fac00c6e1200004e020001fb997007e11b900a3
:101fbc00c109200082804000e0807800a1bf9f0012
:101fcc001fb997007e11b900e10920008280400002
:101fdc00e0807800b1bf9f00bfb8970004015300a8
:101fec000191b90002014200afb897008100d00006
:101ffc008180e900078cb90088804200e2419000a2
:10200c008381fb00f2449000c84cdd008984710090
:10201c001fbd97007e55b900030a20008a8141003c
:10202c006084790013002000081cdd000884ea009d
:10203c0009046400b20490003801980062459000d5
:10204c000a85fb00f2449000c84cdd008904750041
:10205c001fbd97007e55b900280a20000a044400d1
:10206c0060047c00081cdd000884ea00090464009c
:10207c00b204900038019800224590000a85fb00bc
:10208c00b2449000c84cdd00890475001fbd970058
:10209c007e55b900080a20000a04440060047c0044
:1020ac00081cdd000884ea00090464009204900016
:1020bc0018019800224590000a85fb00b24490005c
:1020cc00c84cdd00890475001fbd97007e55b90012
:1020dc00280a20000a04440060047c00081cdd006f
:1020ec000884ea0009046400920490001801980026
:1020fc00424d90000a85fb00d24c9000c84cdd008c
:10210c00890475001fbd97007e55b900080a200090
:10211c000a04440060047c00081cdd000884740080
:10212c00e204900068019800424d90000a85fb0083
:10213c00d24c9000c84cdd00890475001fbd97007f
:10214c007e55b900280a20000a04440060047c0073
:10215c00081cdd0008847400e204900068019800fb
:10216c00f0400a0011880000214190000041eb0072
:10217c00a240980031449000b34098006144900014
:10218c00e24098007141900002c3b300f240980005
:10219c0001499000f0400a000200000082489800bb
:1021ac002149900092c1b300a24898003149900097
:1021bc0092c0b300b24898004149900002c4b300e9
:1021cc00c248980051499000d34898002151900082
:1021dc00f0400a0002000000a2509800415190000b
:1021ec00f0400a0002000000c250980061499000c3
:1021fc00f0400a0002000000e248980001519000f3
:10220c00f0400a00020000008250980061519000da
:10221c00f0400a0002000000e250980001599000c2
:10222c00f0400a00020000008258980021599000ea
:10223c00f0400a0002000000a2589800415990009a
:10224c00f0400a0002000000c2589800615990004a
:10225c00f0400a0002000000e25898000161900072
:10226c00f0400a0002080000826098001fb9970035
:10227c007e14b900420a2000080141006044790034
:10228c0061446400620020000244dd003141900092
:10229c000264a10008417100b240980021619000d5
:1022ac00f0400a0002000000a26098001fb99700dd
:1022bc007e14b900c20a20000801410060017900b7
:1022cc0021149000a210980061619000f0400a0067
:1022dc0002000000e26098001fb997007e14b9005c
:1022ec00620a20000801410060017900411490004d
:1022fc00c210980021699000f0400a000200000012
:10230c00a268980041699000f0400a0002000000a9
:10231c00c268980061699000f0400a000200000059
:10232c00e26898001fb997007e14b900220b2000b8
:10233c000801410060017900011c9000821898008e
:10234c001fb997007e14b900020b20000801410050
:10235c0060017900111c9000921898001fb9970029
:10236c007e14b900420b2000080141006001790085
:10237c00710c9000f208980001619000f0400a0086
:10238c0002080000826098001fb997000200e0006c
:10239c0027003a00314190000234a000b24098006e
:1023ac003141900020030a0002000000b240980066
:1023bc002141900030400a0002000000a240980029
:1023cc002149900020400a0002030000a248980016
:1023dc001fb997007e11b900820ab0006001790024
:1023ec00f1119000f2109800714190000264a0006d
:1023fc00f2409800414190000234a000c240980085
:10240c009fb897008100e80091bf9f005011900089
:10241c009fb89700810f5100e3fe3e000fb8970064
:10242c004f05be004f04be000080fa0000000600fd
:10243c00314190000234a100b2409800314190002b
:10244c0020400a0002030000b24098002141900095
:10245c0030400a0002020000a2409800214990007e
:10246c0020400a0002000000a24898001fb9970003
:10247c007e11b900820ab00060017900f111900060
:10248c00f2109800714190000264a000f240980094
:10249c00414190000234a000c24098009fb89700c0
:1024ac008100e80091bf9f00501190009fb89700e9
:0c24bc00810f5100bcfe3e00d8ff37002d
:020000040000fa
:1024c8000600fa00889fbe008a1f780010002000ce
:1024d800b0bf9f008000eb00c1bf9f000040eb0031
:1024e800c0f79f00c08480000010a100c08488004d
:1024f800c08480000020a100c0848800c0848000bf
:102508000030a100c0848800c08480000040a10081
:10251800c0848800c08480000070a000c084880047
:10252800c08480000090a000c0848800c08480001f
:1025380000e0a000c0848800c084800000f0a100f2
:10254800c0848800a00921000008eb0020002000ba
:10255800e0858800e203200002868800229f200090
:10256800f285880010868800c1bf9f001186800010
:102578004fb89700808f500009003600420c2100a8
:102588000009eb004fb897000000e800c0bf9f00ab
:10259800118680004fb89700808f5000f8ff3e00ea
:1025a800800c21000008eb00640040000008eb00ec
:1025b8000080e9000008eb00640040000008eb0020
:1025c80023002000a389880010002000b08988001b
:1025d800c1002000c1898800d1002000d18988006d
:1025e800c11321008048780009f42100f989880086
:1025f80008fa2000088a880002142000228a88002d
:10260800128a880007902100378a880081022000fa
:10261800418a8800518a8800061e2000668a880040
:1026280004152100000aeb000482e900000aeb000f
:1026380044002000948a8800a08a88009500200021
:10264800b58a880085002000c58a8800aa1521005f
:10265800004d7800e98a8800f88a8800128b880083
:10266800028b8800278b8800318b8800418b88007b
:10267800568b8800f40045008008eb00f200450006
:102688008008eb00848040008048eb00ea8040002e
:1026980080487800e08b8800f08b8800e680400056
:1026a8008008eb00838040008008eb00e109b1005e
:1026b80080487800c0f79f00668140000449780090
:1026c800678140000549780042c1200032878800b0
:1026d80066c0b30005814000064978006b81400060
:1026e8000049eb000281e900cff397000749780021
:1026f80000014100cff397000749780063014100ca
:102708000049eb000201e9000049eb0012ca24006d
:102718009287880032002000a287880072814000da
:102728000009eb009140780061c160000001610080
:102738000411dd00017080000140a10081007100da
:102748000170880061f72f008a8040008048780077
:102758006681400003497800678140000549780098
:1027680002c1200092868800a2c0b3008582400082
:10277800824a7800eb824000804aeb008582e900bb
:10278800804aeb0080824200804aeb00e3824200ec
:10279800804aeb008502e900804aeb0085e52500c8
:1027a800f58688005500200005878800f2824000e1
:1027b800800aeb0091407800e1c2600080826200ec
:1027c800c72add00e17080000170a10081807200dd
:1027d800e1708800e1f92f008a8040008048780085
:1027e800e6824000804aeb00e7824000804aeb0026
:1027f800c5c02000d5878800e8824000864a780056
:10280800eb824000804aeb008582e900804aeb00b9
:1028180080824200804aeb00e3824200804aeb005b
:102828008502e900804aeb00f5ff2700358888001b
:1028380044888800048020005488880091407800eb
:10284800e1c0600000210a00000e000021fb2f00fb
:102858008a8040008048780066824000004a7800fc
:1028680067824000004a7800e4c02000748888002d
:1028780068824000024a78006b8140000049eb0002
:10288800698140000049eb00000141000049eb006c
:10289800630141000049eb000201e9000049eb0037
:1028a80091407800e1c060008080600001814000b4
:1028b800017080000110a100810071000170880082
:1028c80081f82f00848040008008eb00f17c200014
:1028d800f1848800e1f82f00848040008008eb0034
:1028e8008180e9008008eb00f48040008008eb005c
:1028f800713e2000b1858800d3858800d18580008d
:102908000100e00001003a00d08588008000eb005b
:10291800800b21000008eb00e0858000e20f5000ea
:102928000d003200400a21000008eb00f07c200076
:1029380030858800a00a21000008eb00209f2000b5
:10294800408588003fb897004f0578004f04be00c7
:102958000080fa000000060061858800703e2000b3
:102968007085880091858800908580000000e000cf
:1029780002003a001000200090858800e003200043
:1029880080858800400a21000008eb00f07c2000c8
:1029980030858800a00a21000008eb00209f200055
:1029a800408588003fb897004f0578004f04be0067
:0c29b8000080fa0000000600e7ff370076
:020000040000fa
:1029c4000400fa000002780011002000f1bf9f000b
:1029d4001404e00047003200e4409000efcf5000c0
:1029e40048003e0054499000e44090000281fb00fe
:1029f4008180fb008110dd0001007800d02bb7003e
:102a040024499000e44090000281fb008180fb0097
:102a14008110dd0001007800f02bb700144990000c
:102a2400e44090000281fb008180fb008110dd0006
:102a340001007800202bb700e4409000e7cf50005d
:102a44004f003e00e440900081c04000c1ff9f0061
:102a5400e440900002b1200012417800c448900084
:102a64008180fb004ff897008081fb008308dd0024
:102a74008140710002b120000149780002b12000b8
:102a840012417800b44990008381fb004ff897000d
:102a94008080fb008100e8008118dd008140710026
:102aa40002b1200001497800e44090008180fb00dd
:102ab40002b820000448900000f17800f44090002f
:102ac400e1cf500056003200e1cf50005b003900e6
:102ad400e2cf50006a003200e3cf500061003200c0
:102ae4008af0a800344890000004e000010032009d
:102af4008cf0a800ffb89700010078000080fa006d
:102b040000000600644190008000eb00ff4f51007c
:102b1400f9ff3e0054499000e44090000281fb001c
:102b24008180fb00f08050008110dd0001007800fe
:102b3400d22bb70024499000e44090000281fb00ae
:102b44008180fb00f08050008110dd0001007800de
:102b5400f22bb70014499000e44090000281fb007e
:102b64008180fb00f08050008110dd0001007800be
:102b7400222bb700e4409000e7cf5000b1ff3600ad
:102b8400e4409000efcf500033003600e440900062
:102b9400f7cf500041003e00e4409000f0c05000e8
:102ba40081c04000c1ff9f00e440900002b12000ba
:102bb40012417800c44890008180fb004ff89700d0
:102bc4008081fb008308dd008140710002b1200098
:102bd4000149780002b1200012417800b449900004
:102be4008381fb004ff897008080fb008100e800a0
:102bf4008118dd008140710002b120000149780094
:102c0400e44090008180fb0002b82000044890005a
:102c140000f17800f4409000e1cf5000aaff3a00a0
:102c24008a30a800344890000004e000b1ff32006c
:102c34008c30a800ffb89700afff37008a10a800b7
:102c4400344890000004e000aaff32008c10a80071
:102c5400ffb89700a8ff3700e4409000e8c0500098
:102c640079ff37008a70a800344890000004e0001f
:102c7400a0ff32008c70a800ffb897009eff3700b9
:102c84008a50a800344890000004e00099ff320004
:102c94008c50a800ffb8970097ff3700644190005c
:102ca4008000eb00ff4f510093ff3e00e440900092
:082cb400f8c0500064ff370076
:020000040000fa
:102cbc000400fa0012002000e2bf9f008000eb002d
:102ccc00f1bf9f000000e000200032001000e00087
:102cdc0021003d00100190008000eb000200e0009c
:102cec001a0032009000900011017800d000900082
:102cfc0081006100f1bf9f00a00090000100e00086
:102d0c0007003200900090009100780020019000a4
:102d1c009280500001f0a7008100ea00f1bf9f00f3
:102d2c00a8810a0010000000e38f50005b00320005
:102d3c0010003400e58f5000760032006b00350037
:102d4c00e68f50002f0032008000eb00010078006d
:102d5c000080fa0000000600610098001010a1002d
:102d6c001000a100020078000080fa0000000600ac
:102d7c00f9ff3700e18f500052003200e28f500013
:102d8c00f1ff3a0070019000ffb89700810f5100dd
:102d9c006a0036001010a0001018a30024003200a6
:102dac0010017800e10061000104e00020003a000d
:102dbc00e00090008100e800610098006001900044
:102dcc0080089000810f5100090039001000a0000c
:102ddc008008900061009800b00090000100e000b5
:102dec00030032003000900000000100e0bf9f00a3
:102dfc00efb89700010078000080fa000000060090
:102e0c00d5ff370010099000ffb89700810f5100d3
:102e1c00e0ff3e0070019000ffb89700810f510059
:102e2c00dcff39001010a1001018a300dcff3a00e1
:102e3c0010017800e10061000104e0001300320091
:102e4c001018a30011003a00e00090008100e80087
:102e5c006100980060019000a0089000810f510063
:102e6c00e3ff39001000a100a00890006100980059
:102e7c00c00090000100e000ddff32004000900037
:102e8c0000000100e0bf9f00d9ff37008000eb007d
:102e9c0061009800efb89700d6ff370070019000e2
:102eac00ffb89700810f5100baff320070019000fb
:102ebc00ffb89700810f5100b7ff32001010a1002e
:102ecc00d9ff370070019000ffb89700810f5100b7
:102edc00b0ff390010099000ffb89700810f510026
:102eec00adff36001010a100cfff3700700190002d
:102efc00ffb89700810f5100a6ff3a0070019000b7
:102f0c00ffb89700810f5100a3ff3a001010a100e9
:102f1c00c5ff370010099000ffb89700810f5100d2
:102f2c00c0ff310070019000ffb89700810f510075
:102f3c00bcff36001010a00097ff3700100990005e
:102f4c00ffb89700810f510093ff31001010a100c2
:042f5c00b5ff370086
:020000040000fa
:102f60000200fa00881f7800000478000000eb00df
:102f7000e0bf9f00f0000a0018000000600121007f
:102f8000c860900040649800c800de00586190005e
:102f900051649800e8004000686190006164980006
:102fa000c808de00786190007164980061ff22001b
:102fb00008699000016c9800c808de00186990004c
:102fc000116c9800a1ff220028699000216c9800e4
:102fd000c808de0038699000316c980021848000b8
:102fe00038199000311c9800918080004819900099
:102ff000411c98003184800058199000511c9800a1
:103000008180800028199000211c98000180800098
:103010006811900061149800118080007811900070
:10302000711498002180800008199000011c9800fc
:103030003180800018199000111c98008000eb006e
:10304000e1bf9f00486990000281fb00d8689000b2
:10305000c808dd00810071006fb99700828f5000b1
:103060001c003600810021006fb99700efb997006e
:10307000c219dd00838140004211dd0002014000e1
:1030800033197800231178006fb99700efb99700d2
:10309000c219dd00838140004211dd0002014000c1
:1030a0003319780023117800efb997008301e80005
:1030b000e3bf9f00c86990008381fb0058699000be
:1030c0004811dd0002817100efb99700830f5100b4
:1030d000e5ff3e008000eb00e1bf9f0068699000c3
:1030e0000281fb00f8689000c808dd0081007100d3
:1030f0006fb99700828f50002700360021372100da
:103100006fb99700efb99700c219dd0083814000c5
:103110000281e8004211dd0002014000331978000d
:10312000231178006fb99700efb99700c219dd003d
:10313000838140000281e8004211dd00020140006d
:1031400033197800231178006fb99700efb9970011
:10315000c219dd00838140000281e8004211dd00d8
:10316000020140003319780023117800efb997006d
:103170008301e800e3bf9f00e86990008381fb00c2
:10318000786990004811dd0002817100efb9970065
:10319000830f5100daff3e00001c21005c02070093
:1031a000a0808000f8189000701c98004084800077
:1031b000e8189000601c9800100020004f04780070
:0831c0000080fa000000060087
:020000040000fa
:1031c8000200fa008000eb00f1bf9f00f0010a0046
:1031d80010000000e1032100406190004160980068
:1031e8004809de00d0619000526098006881400074
:1031f800e0619000626098004811de00f061900084
:1032080072609800c2fe22008069900002689800ef
:103218004811de00906990001268980002ff2200b1
:10322800a0699000226898004811de00b0699000fb
:103238003268980072848000b019900032189800a3
:10324800e2818000c01990004218980082848000b2
:10325800d019900052189800d2818000a0199000cf
:103268002218980052818000e011900062109800a6
:1032780062818000f01190007210980072818000c5
:10328800801990000218980082818000901990009f
:10329800121898000001eb00f2bf9f00c06990006f
:1032a8008381fb00506990004811dd0002817100a4
:1032b800ffb99700830f51001c003600220321003c
:1032c800ffb997007fba97004222dd00040241004f
:1032d800c219dd0083814000b4197800a411780078
:1032e800ffb997007fba97004222dd00040241002f
:1032f800c219dd0083814000b4197800a411780058
:103308007fba97000402e800f4bf9f00406a90006b
:103318000482fb00d0699000c819dd0083017200a7
:103328007fba9700848f5100e5ff3e000001eb0053
:10333800f2bf9f00e06990008381fb0070699000f4
:103348004811dd0002817100ffb99700830f510019
:1033580027003600e2372100ffb997007fba9700af
:103368004222dd00040241008381e800c219dd0029
:1033780083814000b4197800a4117800ffb9970040
:103388007fba97004222dd00040241008381e800f1
:10339800c219dd0083814000b4197800a4117800b7
:1033a800ffb997007fba97004222dd00040241006e
:1033b8008381e800c219dd0083814000b4197800d8
:1033c800a41178007fba97000402e800f4bf9f00b8
:1033d800606a90000482fb00f0699000c819dd0063
:1033e800830172007fba9700848f5100daff3e0094
:1033f800c02221002e040700100020000080fa00df
:0434080000000600ba
:020000040000fa
:10340c000200fa008000eb00f1bf9f00f0010a00ff
:10341c00100000006106210040619000416098009e
:10342c004809de00d061900052609800688140002d
:10343c00e0619000626098004811de00f06190003d
:10344c007260980022fe2200806990000268980049
:10345c004811de00906990001268980062fe22000c
:10346c00a0699000226898004811de00b0699000b5
:10347c003268980092848000b0199000321898003d
:10348c0022838000c019900042189800a28480000a
:10349c00d01990005218980012838000a019900047
:1034ac002218980092828000e0119000621098001f
:1034bc00a2828000f011900072109800b2828000fd
:1034cc008019900002189800c28280009019900018
:1034dc00121898000001eb00f2bf9f00c069900029
:1034ec008381fb00506990004811dd00028171005e
:1034fc00ffb99700830f51001c003600a205210074
:10350c00ffb997007fba97004222dd000402410008
:10351c00c219dd0083814000b4197800a411780031
:10352c00ffb997007fba97004222dd0004024100e8
:10353c00c219dd0083814000b4197800a411780011
:10354c007fba97000402e800f4bf9f00406a900025
:10355c000482fb00d0699000c819dd008301720061
:10356c007fba9700848f5100e5ff3e000001eb000d
:10357c00f2bf9f00e06990008381fb0070699000ae
:10358c004811dd0002817100ffb99700830f5100d3
:10359c0027003600a2382100ffb997007fba9700a8
:1035ac004222dd00040241008381e800c219dd00e3
:1035bc0083814000b4197800a4117800ffb99700fa
:1035cc007fba97004222dd00040241008381e800ab
:1035dc00c219dd0083814000b4197800a411780071
:1035ec00ffb997007fba97004222dd000402410028
:1035fc008381e800c219dd0083814000b419780092
:10360c00a41178007fba97000402e800f4bf9f0071
:10361c00606a90000482fb00f0699000c819dd001c
:10362c00830172007fba9700848f5100daff3e004d
:10363c0080292100f4030700100020000080fa000c
:04364c000000060074
:020000040000fa
:103650000600fa0010002000d0bf9f000000eb0021
:10366000e0bf9f00f0bf9f00a160800061868800de
:10367000616080002186880071608000318688004a
:10368000e0bf9f00118680006fb89700808f5000c8
:103690000f003600820921006fb8970076004000c5
:1036a00000004000e20078007fb8970000804000f2
:1036b000f0bf9f006fb897000000e800e0bf9f00d8
:1036c000118680006fb89700808f5000f2ff3e0097
:1036d0007fb8970040868800628680000000eb007b
:1036e00021b22000810f5100050036006286800063
:1036f0001000200011032100810f510022003e0024
:1037000061006000c300dd00c08480000030a100c3
:1037100000807000c084880023988000d0988000ca
:1037200082998000319a80000300700002007000ce
:1037300081007000e1806000c708dd00c084800067
:103740000070a10000807000c08488008009210002
:103750004cf40700dfb8970001006000d0bf9f0065
:10376000a9050700d0848000e40f500023003e002c
:103770008099800000f0a100809988005fb89700d0
:103780000080fa00000006000000eb00610060000d
:10379000c300dd00c08480000030a1000080700004
:1037a000c084880023988000d0988000829980008f
:1037b000319a8000030070000200700081007000e8
:1037c000e1806000c708dd00c08480000070a100b7
:1037d00000807000c08488008009210029f407005f
:1037e000dfb8970001006000d0bf9f00860507008a
:1037f000d0848000e40f5000ddff3600708c800024
:10380000a06090008180fb00306090004800dd00e7
:1038100000807000a0998800708c8000904090001b
:1038200077810a0001000000cf08dd008099800048
:1038300000f0a10000807000809988005fb89700b8
:0c3840000080fa0000000600cfff3700f7
:020000040000fa
:10384c000200fa000000eb00f0bf9f000000270010
:10385c00840fb60021003200a1092000800720004f
:10386c000001eb0053f82000804978008149780072
:10387c0082497800207c8000e007b2000000a000a4
:10388c00720520006104200043f820008149780073
:10389c008249780080497800eca10a00840f00006e
:1038ac00a8a00a00840f000080cf50000600320050
:1038bc007fb897008000e800f1bf9f0071382100ad
:1038cc00810f5000f4ff36000000eb00713821002e
:1038dc007fb99700810f51003a003e000000eb00c9
:1038ec0050200a008c0f00001100200050210a000b
:1038fc00860f0000820c2000b0220a00880f000006
:10390c004000200064200a008a0f000020210a00d9
:10391c008a0f00008000eb0098210a008a0f00003b
:10392c00a1092000120020008007200053f820007d
:10393c00804978008149780082497800eca10a001e
:10394c00840f0000a8a00a00840f000080cf500054
:10395c0022003200207c8000e007b2000000a000b2
:10396c00720520006104200043f820008149780092
:10397c008249780080497800eca10a00840f00008d
:10398c00a8a00a00840f000080cf5000060032006f
:10399c007fb897000001e800f2bf9f00713821004a
:1039ac00810f5000f4ff3600eca20a00840f0000d7
:1039bc00a8a10a00840f00000000eb00814f510009
:1039cc00020032000080fa0000000600713821006d
:1039dc007fb99700810f5100faff3e0084efa800d9
:1039ec0084afab0006003a007fb897008000e80077
:1039fc00f1bf9f0071382100810f5000f8ff360095
:103a0c000000eb0084afab00eeff320071382100f8
:103a1c007fb99700810f5100eaff3e0033a00a00e6
:103a2c00840f0000610010000080fa000000060006
:043a3c00e6ff37006a
:020000040000fa
:103a400010f0a6002d0037002014900040159000c3
:103a50008608c3008608c1001201c100301b900017
:103a60000600c8001a039000260598000a0390007b
:103a7000160598001001900092007800002990002f
:103a80000109780010119000928010002019900018
:103a90008208dd0030149000010d78008688c30094
:103aa0008688c1008688c1001281c100401b900039
:103ab0000680c8000000cb000400cd001023900059
:103ac00016a0e60006027800002390001620e6000b
:103ad00006027800100c9000040c7800500c900046
:103ae000040c7800401590000a0390001605980019
:103af000040d7800861d04000000000010019000f5
:103b0000920078000029900001097800000006006a
:103b1000801f7800401090000018eb000008eb00b8
:103b20004f007800801f7800501090000018eb00c4
:103b30000018eb000008eb004f00780000000600c2
:103b4000801f7800811f78005010900001187800c5
:103b50000118780001087800cf0078004f00780045
:103b6000801f7800821f78004010900002187800b3
:103b7000020878004f0178004f007800000006002e
:103b800010f0a6001a003700100190009200780093
:103b90000029900001097800101190009280100017
:103ba000201990008208dd00701b900060199000c1
:103bb000010278001301c1000200c8000400cd001a
:103bc0001023900016a0e600060278000023900063
:103bd0001620e60006027800100c9000040c780015
:103be000500c9000040c7800001e0400000000003f
:103bf00010019000920078000029900001097800df
:043c000000000600ba
:020000040000fa
:103c04000200fa0011002000f1bf9f00a52fa900b7
:103c14002be3a90061e3a90097e3a900cde3a90080
:103c240031002000f0210a000003000021302000b0
:103c340091407800f0400a0001000000223020008a
:103c4400014978004130200091407800f0400a009a
:103c5400010000004230200001497800613020005a
:103c640091407800f0400a0001000000623020001a
:103c7400014978008130200091407800f0400a002a
:103c8400010000008230200001497800a1302000aa
:103c940091407800f0400a0001000000a2302000aa
:103ca40001497800c06091000104e0000300320083
:103cb4003090900051188000501888000cc3bf0049
:103cc400f0400a00000000000ce3b7000ec3bf0080
:103cd400f0400a00000000000ee3b70010c3bf006c
:103ce400f0400a000000000010e3b70012c3bf0058
:103cf400f0400a000000000012e3b70014c3bf0044
:103d0400f0400a000000000014e3b70016c3bf002f
:103d1400f0400a000000000016e3b70018c3bf001b
:103d2400f0400a000000000018e3b7001ac3bf0007
:103d3400f0400a00000000001ae3b7001cc3bf00f3
:103d4400f0400a00000000001ce3b7001ec3bf00df
:103d5400f0400a00000000001ee3b70020c3bf00cb
:103d6400f0400a000000000020e3b70022c3bf00b7
:103d7400f0400a000000000022e3b70024c3bf00a3
:103d8400f0400a000000000024e3b70026c3bf008f
:103d9400f0400a000000000026e3b70028c3bf007b
:103da400f0400a000000000028e3b7007fb8970045
:083db4000080fa000000060087
:020000040000fa
:103dbc0096100000020000008000000004130000b8
:103dcc00580000008000000098100000280100003e
:103ddc00800000007a1000000a0000008000000043
:103dec008a10000004000000800000007213000024
:103dfc000c00000082000000ca720000006f01007d
:103e0c000000a6008e000000c01100006c00000035
:103e1c00800000000010000016000000820000006e
:103e2c000200030000020000030072007100000099
:103e3c008f0e0000000300000300d60054000000a9
:103e4c008410000006000000800000001610000026
:103e5c001400000080000000f62f00000a00000093
:103e6c00800000007e1300000c00000082000000a7
:103e7c002e7d000000cd0e000000a000910000007f
:103e8c002c1200006c000000800000002a100000c2
:103e9c001400000082000000020003000002000079
:103eac000300bd0058000000442700000003000080
:103ebc00050000008e1000000400000080000000cf
:103ecc003e1000001400000080000000ec2f0000e9
:103edc000a000000800000008a1300000c000000a3
:103eec00820000002e7d000000cd0e000000a0001e
:103efc0091000000981200006c000000800000008f
:103f0c0052100000140000008200000002000300a8
:103f1c00000200000300bd00580000004427000010
:103f2c0000030000050000009210000004000000d7
:103f3c0080000000661000001400000080000000eb
:103f4c00e22f00000a0000008000000000000000ca
:020000040000fa
:103f5c000800fa0011002000c1bf9f008000eb0098
:103f6c00d1bf9f00e1bf9f00f1bf9f00d1bf9f0059
:103f7c0050119000dfb89700810f51004e003600b1
:103f8c00a432200005362000848252008582d100a4
:103f9c005fb997007e11b900c109200082804000f2
:103fac00e0807800f1bf9f007fb997000201d0003c
:103fbc000281e9000591b90082004200e1419000c4
:103fcc008381fb00714190004811dd00028171007a
:103fdc000300230002817100b1019000b20098002f
:103fec00814990008381fb00114990004811dd004c
:103ffc000281710033ff2f0003016100c1019000a9
:10400c00c2009800114190000274a00092409800e8
:10401c00414190000234a000c24098001181fb0085
:10402c00914190000278a3000e0032000003e200e0
:10403c00060035006fb997008201e800e3bf9f00ce
:10404c0073382100830f5100f8ff3600efb9970049
:10405c0072382100828f51001a003e0001c3ab0060
:10406c0018003a00814990008381fb0011499000af
:10407c004811dd0002817100c200b300c101900043
:10408c00c20098009140900077810a000100000066
:10409c004fb9970082806000c1bf9f00dfb89700c6
:1040ac008100e800d1bf9f0050119000dfb897004d
:1040bc00810f5100b6ff3e004fb897000080fa0008
:1040cc00000006000000eb000080fa000000060073
:0440dc00fcff3700ae
:020000040000fa
:1040e000889fbe00c90c2100399888008000eb0031
:1040f000419888008082eb00759888004630210046
:10410000f48f2f00160062000090a000000b7800d2
:104110008198880020b22000909888002703200012
:10412000a79888003010b000b0988800481f200081
:10413000c898880063a822005398880042ad2200e6
:1041400062988800a03121001010a0001000a0008b
:1041500016f0a000e9988800f19888002599880059
:10416000100362000680a0000608780031998800dc
:104170002603210046998800579988003610b1001f
:1041800066998800789988000399880012998800b8
:104190001010a0001000a00010f0a0000980e9009d
:1041a000909988006e805400a0998800d599880065
:1041b00000332100100362000680a000060878008a
:1041c000e199880096062000f6998800a60f200045
:1041d000069a8800a6012000169a8800863e2000d4
:1041e000269a8800b3998800c29988001010a1000f
:1041f0001000a10010f0a10064805400409a8800d3
:10420000519a8800859a880060342100100262006b
:104210000480a00004087800919a8800c1662100fb
:10422000a19a8800b79a8800d105b100c19a880088
:10423000017d2000d19a8800639a8800729a8800d4
:104240001010a0001000a00010f0a000100020002e
:084250004f04be00000006004f
:020000040000fa
:104258000200fa0012002000f2bf9f0090029000b6
:1042680003e02000c1e1200083805000058ab900e6
:1042780084804100b00190000300e00028003a006b
:10428800614290000482fb00f1419000c819dd00f2
:1042980083017200200290000411dd000281ea000f
:1042a80003016100b1019000b20098004001900044
:1042b8000200e00027003200214290000482fb0047
:1042c800b1419000c819dd008301720020019000ff
:1042d800140020000221dd0002817100910190008c
:1042e800920098001182fb0091419000c819dd00ee
:1042f8008301720020019000100020000201dd00ff
:104308000281ea0003016100f0020a0011000000c6
:10431800f0bf9f007fb897000080fa0000000600f9
:10432800614290000482fb00f1419000c819dd0051
:1043380083017200200290000411dd0002817100e7
:10434800b1019000b2009800400190000200e00026
:10435800d9ff3a00214290000482fb00b14190004d
:10436800c819dd00830172002001900014002000ac
:104378000221dd000281ea00030161009101900041
:10438800920098001182fb0091419000c819dd004d
:104398008301720020019000100020000201dd005e
:1043a8000281ea0003016100f0020a001100000026
:1043b800f0bf9f007fb897000080fa000000060059
:0443c800d7ff3700e4
:020000040000fa
:1043cc0010f0a60034003700201490004015900027
:1043dc008608c3008608c1001201c100301b900082
:1043ec000600c8001a039000260598000a039000e6
:1043fc00160598001001900092007800002990009a
:10440c0001097800400190008100110010e0a70024
:10441c008100ea0010119000928010002019900089
:10442c008208dd0030149000010d78008688c300ee
:10443c008688c1008688c1001281c100401b900093
:10444c000680c8000000cb000400cd0010239000b3
:10445c0016a0e60006027800002390001620e60065
:10446c0006027800100c9000040c780041a3de00ca
:10447c005024900008054300402490000a0c78005a
:10448c00401590000a03900016059800040d780062
:10449c005a220400000000001001900092007800e5
:1044ac00002990000109780000000600801f7800a8
:1044bc00401090000018eb000008eb004f00780053
:1044cc00801f7800501090000018eb000018eb00d3
:1044dc000008eb004f00780000000600801f7800f9
:1044ec00811f780050109000011878000118780096
:1044fc0001087800cf0078004f007800801f78000a
:10450c00821f780040109000021878000208780092
:10451c004f0178004f0078000000060010f0a60054
:10452c003400370020149000401590008608c3001a
:10453c008608c1001201c100301b90000600c800a3
:10454c001a039000260598000a039000160598009f
:10455c001001900092007800002990000109780069
:10456c00400190008100110010e0a7008100ea00da
:10457c001011900092801000201990008208dd002c
:10458c0030149000010d78008688c3008688c10025
:10459c008688c1001281c100401b90000680c800b3
:1045ac000000cb000400cd001023900016a0e60004
:1045bc0006027800002390001620e6000602780020
:1045cc00100c9000040c780041a3de0050249000e5
:1045dc0008054300402490000a0c78004015900018
:1045ec000a03900016059800040d780008230400b7
:1045fc00000000001001900092007800002990004b
:10460c000109780000000600801f7800401090001f
:10461c000018eb000008eb004f007800801f7800ba
:10462c00501090000018eb000018eb000008eb0095
:10463c004f00780000000600801f7800811f780072
:10464c0050109000011878000118780001087800cb
:10465c00cf0078004f007800801f7800821f780010
:10466c004010900002187800020878004f01780082
:08467c004f0078000000060069
:020000040000fa
:104684000600fa0011002000d1bf9f008000eb005b
:10469400e1bf9f00f1bf9f00e1bf9f005011900058
:1046a400efb89700810f510047003600a332200075
:1046b40004362000030252000482d100efb89700b0
:1046c4007e0bb900c109200086804000e08078009c
:1046d400f1bf9f00ffb897008100d0008180e900fe
:1046e400048bb90086804100e14290008582fb0082
:1046f400714190004811dd00028172000500230021
:1047040002817200b1029000b2009800814a9000c8
:104714008582fb00114990004811dd00028172007e
:1047240035ff2f0005016100c1029000c20098000e
:104734009182fb00114190004811dd00028172005a
:1047440002f0a100f0020a00110000006fb9970006
:104754007e13b900c20a20000601410060017900fd
:10476400a1129000a2109800c14290008582fb0023
:10477400514190004811dd00028172000230a00016
:10478400a1029000a20098001141900001c8b3005a
:10479400814061008180fb008100e900cf08de00d8
:1047a4005fb9970082806000d1bf9f00efb8970087
:1047b4008100e800e1bf9f0050119000efb897001e
:1047c400810f5100bdff3e005fb897000080fa00e2
:0447d40000000600db
:020000040000fa
:1047d8000200fa0010002000f0bf9f00a40fa900fb
:1047e80001eba90001aba9003100200065210a00f6
:1047f800020b000002eba90005eba90005cba900fc
:10480800058ba80071002000a8210a00040b0000f5
:1048180060200a00040b00008100200090210a009b
:10482800060b000007cba90007eba9008000eb00ee
:10483800fd210a00080b0000098ba900096ba900db
:10484800094ba900092ba900090ba90008eba9002d
:1048580008cba90050210a00080b0000fe200a001e
:104868000a0b0000d8210a000a0b00000aeba90075
:104878000a0ba9000a2ba9000c0ba9000c2ba900f4
:1048880010210a000e0b000032200a000e0b000057
:1048980000eca900000ca900002ca900f0002000e1
:1048a800b8200a00020c000002eca900020ca900c2
:1048b800022ca90090210a00d80b000090210a00c0
:1048c800d40b00003100200098210a00d60b00000c
:1048d8000000eb0060200a00d60b000071002000e9
:1048e800ca210a00d60b00003000200098200a00d8
:1048f800da0b00008000eb0060210a00da0b0000f0
:1049080070002000ca200a00da0b00007fb8970068
:084918000080fa000000060017
:020000040000fa
:104920000400fa00881f780018002000d8bf9f00fc
:104930000000eb00e0bf9f00c4fb0700dfb897005a
:1049400001006000d0bf9f004d020700dfb8970054
:1049500001006000d0bf9f00c1020700dfb89700d0
:1049600001006000d0bf9f0021020700dfb8970060
:1049700001006000d0bf9f0023eea800f3020700f3
:10498000dfb8970001006000d0bf9f00cb02070096
:10499000dfb8970001006000d0bf9f0008007800da
:1049a000ad000700dfb8970001006000d0bf9f0096
:1049b00076020700dfb8970001006000d0bf9f00bb
:1049c00042010700dfb8970001006000d0bf9f00e0
:1049d000c3fd0700dfb8970001006000d0bf9f0053
:1049e0000000eb0064200a00400800000028a90035
:1049f0002028a90001e1a800000880004f00de0087
:104a0000dfb8970001006000d0bf9f0023eea9002f
:104a10005fb897000000e00001003a000000fe00cf
:104a20000028ab0006003a006fb897008000e8004d
:104a3000e1bf9f00f1522700810f5000f8ff3600c0
:104a40000028a9000000eb00e0bf9f0023eea800b3
:104a5000fffa07006802070023eea900000000002b
:044a6000efff37002d
:020000040000fa
:104a64000600fa0011002000d1bf9f008000eb0077
:104a7400e1bf9f00e1bf9f0050119000efb8970085
:104a8400810f510036003600a43220000536200084
:104a9400848252008582d1006fb997007e11b900db
:104aa400c109200082804000e0807800f1bf9f00af
:104ab4007fb997000201d0000281e9000591b90095
:104ac40082004200e14190008381fb00714190002b
:104ad4004811dd000281710003002300028171008e
:104ae40031039000b200980041619000f0400a0048
:104af40002000000c2609800414390000683fb005e
:104b0400514190004811dd00020173000230a00001
:104b140021039000a2009800614190000281fb00f3
:104b2400f1409000c808dd008100710083816000bd
:104b34008301ea00cf19de00dfb8970081816100ac
:104b4400d3bf9f00efb897008100e800e1bf9f004a
:104b540050119000efb89700810f5100ceff3e0036
:0c4b64005fb897000080fa000000060017
:020000040000fa
:104b70000600fa0011002000d1bf9f008000eb006a
:104b8000e1bf9f00f1bf9f00e1bf9f005011900067
:104b9000efb89700810f51002c003600a33220009f
:104ba00004362000030252000482d100efb89700bf
:104bb0007e0bb900c109200086804000e0807800ab
:104bc000f1bf9f00ffb897008100d0008180e9000d
:104bd000048bb90086804100414190000234a0005e
:104be000c2409800e14290008582fb007141900034
:104bf0004811dd0002817200f5ff2c000501610003
:104c0000b1029000b200980061419000f140900024
:104c1000c808dd0002002300828060008100e900f6
:104c2000cf08de005fb9970082806000d1bf9f008f
:104c3000efb897008100e800e1bf9f00501190009d
:104c4000efb89700810f5100d8ff3e005fb8970082
:084c50000080fa0000000600dc
:020000040000fa
:104c58000400fa00f0bf9f0012002000e2bf9f008e
:104c68007fb8970081c8200084c920000102520043
:104c78000000e90000a2b9000480400090409000c4
:104c88000174a10011409800a040900001ceb3002b
:104c980021409800b0419000c1cfb30081c06100ad
:104ca8000104a000314098009040900065400a003f
:104cb8000100000011409800904090000124a100dc
:104cc80011409800904090000104a1001140980004
:104cd8001064a10053400a00100000001024a10035
:104ce80010400a0010000000904090000114a0003d
:104cf80011409800e040900080c0eb0061409800af
:104d0800f040900071c0b300714098007fb89700e0
:104d18000000e9000011dd00b28488006fb8970038
:084d28000080fa000000060003
:020000040000fa
:104d30000200fa00881f780018002000e8bf9f00da
:104d400080092100affb0700efb897000100600069
:104d5000e0bf9f008009210084f40700efb89700ae
:104d600001006000e0bf9f009bfe0700efb89700c6
:104d700001006000e0bf9f00400e210011f7070016
:104d8000efb8970001006000e0bf9f00000d210018
:104d90000cf70700efb8970001006000e0bf9f002c
:104da000800f210007f70700efb8970001006000af
:104db000e0bf9f00c010210002f70700efb8970086
:104dc00001006000e0bf9f0000122100fdf6070017
:104dd000efb8970001006000e0bf9f00800921004c
:104de0004a010700efb8970001006000e0bf9f0094
:104df00032280a000e0b00006fb897004f047800ad
:084e00000080fa00000006002a
:020000040000fa
:104e0800d0848000e20f500001003200000006004c
:104e1800c08480000048a300fcff3a00c0848000e2
:104e28000018a300f9ff32007a30ec00d08380002c
:104e3800e70f50001a003600e083800021868000ca
:104e480000804000e0838800008480003186800074
:104e58000080400000848800e08380004300de007a
:104e6800e0838800008480004300de00008488001e
:104e7800108d8000e183800040019000410098007f
:104e8800b08d8000018480004001900041009800ae
:104e9800c08480000040a000c08488000000060094
:104ea800e08380002186800000804000e083880045
:104eb80000848000318680000080400000848800e3
:044ec80000000600e0
:020000040000fa
:104ecc000200fa0010002000f0bf9f007bf50700e5
:104edc00ffb8970001006000f0bf9f0057f107007a
:104eec00ffb8970001006000f0bf9f008dff070026
:104efc00ffb8970001006000f0bf9f0080092100ff
:104f0c0013fc0700ffb8970001006000f0bf9f0082
:104f1c007fb897000000e00003003200c0848000de
:104f2c000020a000c08488000f000700ffb8970085
:104f3c0001006000f0bf9f00f00ba80050002000a3
:104f4c00ec200a006c0800000b68a9002b68a80074
:104f5c00c084800000f0a000c08488007fb8970057
:084f6c000080fa0000000600bd
:020000040000fa
:104f74000600fa0010002000d0bf9f000000eb00e4
:104f8400e0bf9f00f0bf9f0001eba8008a10f8006b
:104f9400000cf900508480004800dd008a10b7003e
:104fa400f0bf9f00036080007fb997006fb897003f
:104fb4008000e800e1bf9f0071382100810f50009c
:104fc4000a0036006fb997000000eb007138210029
:104fd400810f510003003e008a10f8000a0bf9000b
:104fe4005fb897000080fa0000000600828f51002d
:104ff400f4ff3200036080007fb997006fb8970018
:105004008000e800e1bf9f0071382100810f50004b
:08501400ecff3e00f5ff370040
:020000040000fa
:10501c000200fa0012002000f2bf9f0090029000e4
:10502c0003e02000c1e1200083805000058ab90014
:10503c0084804100b00190000300e0000e003200bb
:10504c00614290000482fb00f1419000c819dd0020
:10505c0083017200200090000011dd000281ea0043
:10506c000301610031009000b20098007fb89700f6
:10507c000080fa0000000600614290000482fb00f0
:10508c00f1419000c819dd008301720020009000ee
:10509c000011dd000281710031009000b200980017
:1050ac007fb897000080fa0000000600f2ff37007e
:020000040000fa
:1050bc000200fa0012002000f2bf9f009002900044
:1050cc0003e02000c1e1200083805000058ab90074
:1050dc0084804100b00190000300e0000d0032001c
:1050ec00614290000482fb00f1419000c819dd0080
:1050fc0083017200200090000011dd00028171001c
:10510c0031009000b20098007fb897000080fa0040
:10511c0000000600614290000482fb00f141900007
:10512c00c819dd0083017200200090000011dd0021
:10513c000281ea000301610031009000b200980086
:10514c007fb897000080fa0000000600f1ff3700de
:020000040000fa
:10515c000200fa0011c0b300e1ff9f009001900023
:10516c0001e02000c2e12000010151000391b900cf
:10517c0002814000c24190008381fb0052419000ab
:10518c004811dd0002817100a00090001300200086
:10519c008118dd008280600001f0a7008100ea0028
:1051ac008100ea00cf08de00e1ff9f003000900094
:1051bc00830f5000030032006ff897000080fa0054
:1051cc0000000600eff897000180fb000080510002
:1051dc00e0ff9f006ff897000080fa0000000600c7
:0451ec00f8ff370091
:020000040000fa
:1051f0000200fa0010002000f0bf9f00002eef0018
:105200001c2eef0023cea9001fcea90023eea9007b
:105210001feea900234ea9001f4ea900230ea900ce
:105220001f0ea900232ea9001f2ea9000000eb00cd
:1052300051052000b1468800a10a2000b14688002f
:105240000068880020022000d8200a00880d000095
:105250003102200050210a00880d0000008020004b
:1052600051052000b1468800a10a2000b1468800ff
:10527000006888007fb897000080fa0000000600f0
:020000040000fa
:105280000200fa000000eb00f0bf9f008fefa900c2
:105290003100200098210a00920f00001000200029
:1052a00050200a008e0f0000d1072000b0210a0014
:1052b000900f00002000200064200a00920f0000e0
:1052c0001100200020210a00920f00008f0fa8007b
:1052d0008fefa8000000eb008e0fe20009003d00f8
:1052e0008fcfab0006003a007fb897008000e8003f
:1052f000f1bf9f0071382100810f5000f8ff360088
:0c530000100020000080fa0000000600f1
:020000040000fa
:10530c000200fa00881f78000004780010002000ca
:10531c00e0bf9f0008d891000004e00010003a00a4
:10532c0028e091000004e00004003a006fb89700f8
:10533c004f0478000080fa0000000600200e2000c8
:10534c0008004000c1fb0700e0bf9f006fb897004a
:10535c004f0478000080fa0000000600f7ff3700c9
:10536c00800d200008004000b8fb0700e0bf9f0044
:10537c0028e091000004e000ecff3200efff370062
:020000040000fa
:10538c000200fa0010002000f0bf9f00b1848000e2
:10539c00cf08dd004064800000f0a10000807000a8
:1053ac004064880011a10a0096100000cf08dd00af
:1053bc00c064800000f0a10000807000c064880010
:1053cc0022a10a0096100000cf08dd004065800085
:1053dc0000f0a100008070004065880081eca800fe
:0c53ec007fb897000080fa000000060067
:020000040000fa
:1053f8000200fa0010002000f0bf9f00403021009a
:105408002cf60700ffb8970001006000f0bf9f006e
:10541800a031210027f60700ffb8970001006000bf
:10542800f0bf9f000033210022f60700ffb8970065
:1054380001006000f0bf9f00603421001df60700e6
:10544800ffb8970001006000f0bf9f007fb8970089
:085458000080fa0000000600cc
:020000040000fa
:1054600001e1a90001a1a9000181a9000161a90030
:105470000141a9003000200098200a00000100002e
:1054800000e1a9000000eb0054200a000001000028
:105490000041a9000021a9000421ef00f0702200c2
:1054a000400888000000eb0064200a00400800006b
:0c54b0000028a9002028a9001000050019
:020000040000fa
:1054bc000200fa0010002000f0bf9f0081eca90050
:1054cc0081aca9002100200076210a00800c00008c
:1054dc0054200a00800c00008000eb0020210a0000
:1054ec00800c000090200a00840c000090200a0020
:1054fc00860c00007fb897000080fa0000000600c0
:020000040000fa
:10550c000200fa00881f780018002000e8bf9f00f6
:10551c008009210050fd0700efb8970001006000e2
:10552c00e0bf9f00800921001070a000d884880083
:10553c006fb897004f0478000080fa000000060056
:020000040000fa
:10554c000200fa0010002000f0bf9f00dde8a90067
:10555c00dc08a900dc28a800de08a800de28a800ca
:10556c00de48a800dde8a8007fb897000080fa00ac
:04557c000000060025
:020000040000fa
:10558000009b8800203621001008e8000000000081
:10559000000000000000000000000000000000000b
:0855a0000000000000000600fd
:020000040000fa
:1055a8000200fa000000eb00f0bf9f00100020008e
:1055b800d08488008009210010f0a0007fb89700ef
:0855c8000080fa00000006005b
:020000040000fa
:04be0000ffff000040
:020000040000fa
:04be2000ffffff0021
:020000040000fa
:04be30007fffff0091
:020000040000fa
:04be38007be7ff00a5
:020000040000fa
:04be4000677fff0019
:020000040000fa
:04be4800ffffff00f9
:020000040000fa
:04be5000ddffff0013
:020000040000fa
:04be58000000ff00e7
:020000040000fa
:04be60000000ff00df
:020000040000fa
:04be68000000ff00d7
:020000040000fa
:04be70000000ff00cf
:020000040000fa
:04be7800ffffff00c9
:020000040000fa
:04be8000fffcff00c4
:020000040000fa
:04be8800c9ffff00ef
:00000001FF
